:020000000029D5
:020008000800EE
:100010001330840005309000FE30910011088600F6
:1000200066000608E0398000800E0310800C050889
:100030009200120D083980040F3080060314910DD0
:10004000840A900B0E2800341A308400053090008A
:10005000FD306500000000000000FC306500083045
:100060009100800D03183828FC3065004E203B2895
:10007000FE3065004E20910B3128FE3065004E2089
:10008000800D840A900B2F28FC306500FD30650040
:10009000000000000000FF306500003401386500FA
:1000A000000000000000FE3965000034F630000753
:1000B000031C5C28093080000034100803196828EC
:1000C00012089C0703189B0A11089B0790035D28E0
:1000D00000342A202A202A20202075205F2050204A
:1000E0004C204C20202031202E2031202020302078
:1000F00038202E20302033202E203920362020207A
:100100004420462031204F20472020202A202A202A
:100110002A20202031202E2031202E203120362070
:100120004620382034202020312035202E20302039
:1001300037202E203020322020204F20452039200B
:0E0140004D204B20562020202A202A202A2045
:1002000083120313FC30850093019401950196013C
:10021000970198019901990308201730840000087C
:100220009800033980000430980584035620840325
:100230005620840356208403181920295620262985
:10024000F8300007031C2629073080001330840093
:1002500003010007840A0007840A0007840A0007D4
:10026000840A0007840A0007840A800680000319B4
:100270000C299B0113089C0018195B291408900095
:10028000003091000A3092005D2015089000003087
:100290009100643092005D201608900003309100B8
:1002A000E83092005D201708900027309100103050
:1002B00092005D20772914089000003091000830EA
:1002C00092005D201508900000309100503092009F
:1002D0005D201608900003309100203092005D20D0
:1002E000170890001F309100403092005D20C2300E
:0E02F0009A00C6309D0000309E0024200C298C
:00000001FF
